:040000000227592258
:10000B000233577B017A02791612352E90021A743D
:10001B00E0F07F011234C62202260EE709F608DF54
:10002B00FA8046E709F208DFFA803E88828C83E784
:10003B0009F0A3DFFA8032E309F608DFFA8078E3F0
:10004B0009F208DFFA807088828C83E309F0A3DF62
:10005B00FA806489828A83E0A3F608DFFA805889E4
:10006B00828A83E0A3F208DFFA804C80D280FA8088
:10007B00C680D4806980F28033801080A680EA80AD
:10008B009A80A880DA80E280CA803389828A83ECE6
:10009B00FAE493A3C8C582C8CCC583CCF0A3C8C56A
:1000AB0082C8CCC583CCDFE9DEE7800D89828A83E9
:1000BB00E493A3F608DFF9ECFAA9F0EDFB228982B1
:1000CB008A83ECFAE0A3C8C582C8CCC583CCF0A365
:1000DB00C8C582C8CCC583CCDFEADEE880DB898269
:1000EB008A83E493A3F208DFF980CC88F0EF6001F8
:1000FB000E4E60C388F0ED2402B4040050B9F582B3
:10010B00EB2402B4040050AF2323458223900076E6
:10011B0073BB010689828A83E0225002E722BBFE71
:10012B0002E32289828A83E49322BB010CE58229B4
:10013B00F582E5833AF583E0225006E92582F8E65D
:10014B0022BBFE06E92582F8E222E58229F582E54B
:10015B00833AF583E49322BB010FF8E58229F582FC
:10016B00E5833AF583E028F0225009C58229F8E5AA
:10017B008226F622BBFE09C58229F8E22582F222ED
:10018B00F8EA2583F583E9932822BB010689828A45
:10019B0083F0225002F722BBFE01F322F8BB010DC4
:1001AB00E58229F582E5833AF583E8F0225006E9EA
:1001BB002582C8F622BBFE05E92582C8F222EF8D07
:1001CB00F0A4A8F0CF8CF0A428CE8DF0A42EFE22A4
:1001DB00BC000BBE0029EF8DF084FFADF022E4CC08
:1001EB00F875F008EF2FFFEE33FEEC33FCEE9DECD1
:1001FB00984005FCEE9DFE0FD5F0E9E4CEFD22ED17
:10020B00F8F5F0EE8420D21CFEADF075F008EF2F60
:10021B00FFED33FD4007985006D5F0F222C398FD51
:10022B000FD5F0EA22C2D5EC30E709B2D5E4C39D75
:10023B00FDE49CFCEE30E715B2D5E4C39FFFE49ED2
:10024B00FE1201DBC3E49DFDE49CFC80031201DB89
:10025B0030D507C3E49FFFE49EFE22C5F0F8A3E070
:10026B0028F0C5F0F8E582158270021583E038F0AE
:10027B0022A3F8E0C5F025F0F0E582158270021597
:10028B0083E0C838F0E822BB010A89828A83E0F553
:10029B00F0A3E022500687F009E71922BBFE07E323
:1002AB00F5F009E3192289828A83E493F5F074014E
:1002BB009322BB0110E58229F582E5833AF583E0B1
:1002CB00F5F0A3E0225009E92582F886F008E62232
:1002DB00BBFE0AE92582F8E2F5F008E222E5832A63
:1002EB00F583E993F5F0A3E99322F8BB0111E582BD
:1002FB0029F582E5833AF583E8F0E5F0A3F0225087
:10030B0009E92582C8F608A6F022BBFE09E9258279
:10031B00C8F2E5F008F222EF2BFFEE3AFEED39FDC5
:10032B00EC38FC22C3EF9BFFEE9AFEED99FDEC98A7
:10033B00FC22E88FF0A4CC8BF0A42CFCE98EF0A46B
:10034B002CFC8AF0EDA42CFCEA8EF0A4CDA8F08B4B
:10035B00F0A42DCC3825F0FDE98FF0A42CCD35F091
:10036B00FCEB8EF0A4FEA9F0EB8FF0A4CFC5F02E22
:10037B00CD39FEE43CFCEAA42DCE35F0FDE43CFC8B
:10038B002275F008758200EF2FFFEE33FECD33CDD3
:10039B00CC33CCC58233C5829BED9AEC99E5829820
:1003AB00400CF582EE9BFEED9AFDEC99FC0FD5F01F
:1003BB00D6E4CEFBE4CDFAE4CCF9A88222B800C196
:1003CB00B90059BA002DEC8BF084CFCECDFCE5F003
:1003DB00CBF97818EF2FFFEE33FEED33FDEC33FC4A
:1003EB00EB33FB10D703994004EB99FB0FD8E5E4F3
:1003FB00F9FA227818EF2FFFEE33FEED33FDEC33D5
:10040B00FCC933C910D7059BE99A4007EC9BFCE963
:10041B009AF90FD8E0E4C9FAE4CCFB2275F010EF9F
:10042B002FFFEE33FEED33FDCC33CCC833C810D7E2
:10043B00079BEC9AE899400AED9BFDEC9AFCE89936
:10044B00F80FD5F0DAE4CDFBE4CCFAE4C8F922C31B
:10045B00E49FFFE49EFEE49DFDE49CFC22EB9FF5F4
:10046B00F0EA9E42F0E99D42F0EC6480C86480980B
:10047B0045F022EB9FF5F0EA9E42F0E99D42F0E851
:10048B009C45F022E8600FECC313FCED13FDEE135B
:10049B00FEEF13FFD8F122E8600FEFC333FFEE330B
:1004AB00FEED33FDEC33FCD8F122BB010789828AC8
:1004BB00830205435005E9F80206E9BBFE05E9F89E
:1004CB000206F589828A8302054FBB010DE582295D
:1004DB00F582E5833AF5830205435007E92582F857
:1004EB000206E9BBFE07E92582F80206F5E582293B
:1004FB00F582E5833AF58302054FBB010789828AB2
:10050B00830205E05005E9F802071BBBFE05E9F87D
:10051B0002072722BB010DE58229F582E5833AF517
:10052B00830205E05007E92582F802071BBBFE0793
:10053B00E92582F802072722E0FCA3E0FDA3E0FEF9
:10054B00A3E0FF22E493FC740193FD740293FE7409
:10055B000393FF22E0F8A3E0F9A3E0FAA3E0FB2268
:10056B00E493F8740193F9740293FA740393FB22E6
:10057B00BB010DE58229F582E5833AF58302055F20
:10058B005007E92582F8020701BBFE07E92582F82F
:10059B0002070EE58229F582E5833AF58302056BA6
:1005AB007401FF3395E0FEFDFCA3A3A3E0CF2FF076
:1005BB00E582158270021583E0CE3EF0E58215824E
:1005CB0070021583E0CD3DF0E58215827002158334
:1005DB00E0CC3CF022ECF0A3EDF0A3EEF0A3EFF0B7
:1005EB0022A8828583F0D083D082120603120603E1
:1005FB00120603120603E473E493A3C583C5F0C587
:10060B0083C8C582C8F0A3C583C5F0C583C8C5829E
:10061B00C822BB010789828A830205EC5005E9F8E1
:10062B00020733BBFE05E9F802074C22E0FBA3E00F
:10063B00FAA3E0F922F8E0FBA3A3E0F925F0F0E53B
:10064B0082158270021583E0FA38F022EBF0A3EAF0
:10065B00F0A3E9F022BB010DE58229F582E5833A8F
:10066B00F5830206375007E92582F8020765BBFEC2
:10067B0007E92582F802076EE58229F582E5833AC0
:10068B00F583020777D083D082F8E493701274015C
:10069B0093700DA3A393F8740193F5828883E4738D
:1006AB007402936860EFA3A3A380DF8A838982E43B
:1006BB0073EC8EF0A4CCC5F0CCCDF8EFA4CEC5F086
:1006CB002DFDE43CFCE8A42EC8C5F03DFDE43CFC4C
:1006DB00EFA4FFE5F028FEE43DFDE43CFC22E6FC44
:1006EB0008E6FD08E6FE08E6FF22E2FC08E2FD084C
:1006FB00E2FE08E2FF22E6FB08E6F908E6FA08E666
:10070B00CBF822E2FB08E2F908E2FA08E2CBF82286
:10071B00ECF608EDF608EEF608EFF622ECF208ED33
:10072B00F208EEF208EFF222D083D082E493F608BF
:10073B00740193F608740293F608740393F6740429
:10074B0073D083D082E493F208740193F20874029D
:10075B0093F208740393F2740473E6FB08E6FA0849
:10076B00E6F922E2FB08E2FA08E2F922E493FB74D1
:10077B000193FA740293F9229004C612065790045F
:10078B00C6120637758204758300120135FFEF120E
:10079B0006900886540E3C550C8D560D7E570A3428
:1007AB008308E493095C9407BFE00DA2E10DDBE93C
:1007BB0000000E3C9004C612063775820B75830041
:1007CB00E41201A79004C612063775820A758300DE
:1007DB00E41201A77F0012203B7BFF7A28798AC0A5
:1007EB0003C002C0019004C61206377582067583DA
:1007FB0000120660758201758300120135FF7E00C1
:10080B009002ABEEF0A3EFF0D001D002D0031212A6
:10081B00387F0012203B9004C6120637758209758B
:10082B00830074011201A79004C612063775820566
:10083B0075830074541201A79004C6120637758293
:10084B000475830074E11201A79002D0120543EFE7
:10085B00247DFFEE3400FEED3400FDEC3400FC9003
:10086B0004C6120637120505229004C61206377508
:10087B00820475830074541201A7229004C61206D9
:10088B0037758206758300120660758201758300C9
:10089B00120135FF12310AEF6003020E3C9004C6C1
:1008AB001206377582067583001206607582017514
:1008BB008300120135FF9004C6120637E9240CF9A8
:1008CB00EA3400FA1226B79004C612063775820472
:1008DB0075830074931201A7229004C61206377514
:1008EB00820C7583001204D51232CF9004C6120607
:1008FB0037758210758300EE8FF01202F59004C6E7
:10090B0012063775820675830012066075820475B0
:10091B0083001202BDFFAEF09004C612063775823B
:10092B00107583001202BDFDACF0122BAD9004C606
:10093B00120637758212758300EE8FF01202F59056
:10094B0004C612063775820475830074941201A7CE
:10095B00229004C61206377582267583001202BDDB
:10096B00FFAEF09004C6120637758224758300EE35
:10097B008FF01202F59004C6120637758228758324
:10098B00001202BDFFAEF09004C612063775822628
:10099B00758300EE8FF01202F59004C612063775C0
:1009AB0082127583001202BDFFAEF09004C61206D0
:1009BB0037758228758300EE8FF01202F59004C60E
:1009CB00120637E92424F9EA3400FA12213790048D
:1009DB00C61206377582267583001202BDFFAEF074
:1009EB009004C6120637758214758300EE8FF012D1
:1009FB0002F59004C6120637758209758300120141
:100A0B0035FFEF60129004C61206377582047583AA
:100A1B000074831201A7229004C612063775820454
:100A2B0075830074561201A7229004C612063775FF
:100A3B00820B758300120135FFEFC3940C502A7D96
:100A4B00397F0012365F9004C612063775820B751C
:100A5B00830074011201629004C61206377582047A
:100A6B0075830074541201A7229004C612063775C1
:100A7B00820675830012066075820275830012026E
:100A8B00BDFFAEF09004C612063775821075830059
:100A9B001202BDFDACF0122D1F9004C61206377565
:100AAB008206758300120660758204758300EE8FD3
:100ABB00F01202F57F0012203B7BFF7A2879A612F9
:100ACB0012387F0012203B7BFF7A2879BEC003C00F
:100ADB0002C0019004C61206377582067583001298
:100AEB000660758201758300120135FF7E0090024E
:100AFB00ABEEF0A3EFF09004C612063775821075BB
:100B0B0083001202BDFFAEF09002ADEEF0A3EFF04A
:100B1B009004C6120637758206758300120660753F
:100B2B0082047583001202BDFFAEF09002AFEEF0AF
:100B3B00A3EFF09004C61206377582067583001278
:100B4B0006607582027583001202BDFFAEF0900243
:100B5B00B1EEF0A3EFF0D001D002D0031212387F28
:100B6B000012203B7BFF7A2879EBC003C002C00147
:100B7B009004C612063775820675830012066075DF
:100B8B008201758300120135FF7E009002ABEEF0FF
:100B9B00A3EFF09004C6120637758210758300120E
:100BAB0002BDFFAEF09002ADEEF0A3EFF09004C6E5
:100BBB0012063775820675830012066075820475FE
:100BCB0083001202BDFFAEF09002AFEEF0A3EFF088
:100BDB009004C6120637758206758300120660757F
:100BEB0082027583001202BDFFAEF09002B1EEF0EF
:100BFB00A3EFF0D001D002D0031212389004C6122A
:100C0B0006377582147583001202BDFFAEF0E4FC4B
:100C1B00FD9004C612063775821675830012051FE8
:100C2B009004C6120637758206758300120660752E
:100C3B008206758300120135F9C0019004C61206B5
:100C4B00377582167583001204D5D001A8011204E2
:100C5B00A29004C612063775821A75830012051FFF
:100C6B009004C6120637758209758300E41201A73A
:100C7B009004C612063775820475830074561201F0
:100C8B00A7229004C6120637E9241AF9EA3400FAAF
:100C9B00C003C002C0011204B59004C6120637751A
:100CAB00821675830012057B12032FD001D002D060
:100CBB00031205059004C6120637E9241AF9EA3423
:100CCB0000FAC003C002C0011204B5C004C005C0C5
:100CDB0006C0079004C6120637758214758300127E
:100CEB0002BDFFAEF0AB07AA06E4F9F8D007D006B9
:100CFB00D005D004120322D001D002D00312050577
:100D0B009004C6120637758206758300120660754D
:100D1B008206758300120135F9C0019004C61206D4
:100D2B003775821A7583001204D5D001A8011204FD
:100D3B008F9004C612063775821675830012051F35
:100D4B009004C61206377582167583001204D5906F
:100D5B0004C6120637758222758300EE8FF01202DD
:100D6B00F59004C61206377582047583007457120A
:100D7B0001A7229004C612063775820A7583007488
:100D8B00011201A79004C612063775820475830001
:100D9B0074541201A722229004C61206371204B50E
:100DAB009002D012055FC312047E5003020E3C90DA
:100DBB0004C6120637758205758300120135FF9044
:100DCB0004C6120637758204758300EF1201A72241
:100DDB009004C61206371204B57BFF7AFF79FF78B1
:100DEB00FF1203229004C61206371205059004C6A3
:100DFB001206371204B57B007A0079007800C31213
:100E0B00047E702D9004C612063712061D000000DA
:100E1B00009004C6120637758205758300120135E2
:100E2B00FF9004C6120637758204758300EF12011A
:100E3B00A7229004C01206577B017A01794E120744
:100E4B00837B017A01797C1207837B017A0179AA72
:100E5B001207837B017A0179D81207839004C012A1
:100E6B000637758204758300120135FFEF12069069
:100E7B000F360B10420D0EF20E11200F0FC0161075
:100E8B00632D0E9AE01132E1116BE9000011CC7F5A
:100E9B000012203B9004C012063775822575830023
:100EAB00E41201A79004C0120637758226758300E1
:100EBB00E41201A79004C012063775822A758300CD
:100ECB00E475F0001202F57F0012203B7BFF7A2FB6
:100EDB0079331212389004C0120637758204758369
:100EEB0000740E1201A7229001E2E0FFEF64016093
:100EFB00030211CC900158E4F0900186E4F09001CC
:100F0B00B4E4F09001E2E4F09004C012063775826D
:100F1B002575830074011201629004C012063775A7
:100F2B008204758300740B1201A7229004C0120671
:100F3B0037758225758300120135FFEFC39401408D
:100F4B00629004C0120637758225758300E4120186
:100F5B00A7900170E0FEA3E0FF90017AEEF0A3EF03
:100F6B00F090019EE0FEA3E0FF9001A8EEF0A3EF4E
:100F7B00F09001CCE0FEA3E0FF9001D6EEF0A3EFE2
:100F8B00F09001FAE0FEA3E0FF900204EEF0A3EF75
:100F9B00F09004C012063775820475830074161224
:100FAB0001A7229004C01206377582047583007462
:100FBB000E1201A72290017AE0FEA3E0FFE4FCFDF4
:100FCB009002271205E090022712055F9001A8E01E
:100FDB00FEA3E0FFE4FCFD1203229002271205E0C2
:100FEB0090022712055F9001D6E0FEA3E0FFE4FC20
:100FFB00FD1203229002271205E090022712055FD3
:10100B00900204E0FEA3E0FFE4FCFD120322900239
:10101B00271205E0900227120543780212048F90E5
:10102B00022F1205E09004C01206377582047583F7
:10103B0000740D1201A72290022F12054390022378
:10104B001205E0121B699004C012063775820475F5
:10105B008300742D1201A722900240E0FEA3E0FF53
:10106B0090023EE0FCA3E0FDD3ED9FEC9E403F9051
:10107B0004C012063775822A7583001202BDFFAEBB
:10108B00F09004C01206377582287583001202BDDA
:10109B00FDACF0C3ED9FFFEC9EFE9004C012063733
:1010AB0075822C758300EE8FF01202F5801390047D
:1010BB00C012063775822C758300E475F00012029E
:1010CB00F59004C0120637758205758300740E12F5
:1010DB0001A79004C012063775820475830074E172
:1010EB001201A79002D0120543EF2411FFEE34003A
:1010FB00FEED3400FDEC3400FC9004C012063712F8
:10110B000505229004C0120637758204758300749E
:10111B000E1201A7229004C0120637758204758344
:10112B0000740E1201A7229004C01206371204B5E8
:10113B009002D012055FC312047E50030211CC90B3
:10114B0004C0120637758205758300120135FF90B6
:10115B0004C0120637758204758300EF1201A722B3
:10116B009004C01206371204B57BFF7AFF79FF7823
:10117B00FF1203229004C01206371205059004C01B
:10118B001206371204B57B007A0079007800C3127F
:10119B00047E702D9004C012063712061D0000004D
:1011AB00009004C012063775820575830012013555
:1011BB00FF9004C0120637758204758300EF12018D
:1011CB00A722E50824ABF582E43402F583E0050899
:1011DB00229002A83007039002ABE475F0011206CF
:1011EB004002011C2000E97F2ED2008018EF540F23
:1011FB002490D43440D4FF30040BEF24BFB41A0036
:10120B0050032461FFE50960021509050CE50C701C
:10121B0002050B30070E9002A8E475F00112064090
:10122B00EF0201950236987403D2078003E4C207DC
:10123B00F5089002A8120657E4F509F50BF50CE535
:10124B000960077F2012121080F5750AFFC201C2D8
:10125B0000C202C203C205C206C2081211DCFF7033
:10126B000D3007057F00121221AF0CAE0B22B425F7
:10127B005FC2D5C2041211DCFF24D0B40A00501A8D
:10128B0075F00A780930D50508B6FF0106C6A42605
:10129B00F620D5047002D20380D924CFB41A00EF04
:1012AB005004C2E5D204021422D20180C6D20080BF
:1012BB00C0D20280BCD2D580BAD20580B47F2012B6
:1012CB0012102002077401B5090040F11211CDFF75
:1012DB0012121002124AD208D20680951211CDFBBF
:1012EB001211CDFA1211CDF94A4B700679F37A141B
:1012FB007BFF20022EE509602A7E008E827583001B
:10130B0012013560060EEE650A70F0C2D5EBC0E037
:10131B00EAC0E0E9C0E0EE121469D0E0F9D0E0FADF
:10132B00D0E0FB12011CFF60AAEBC0E0EAC0E0E9D1
:10133B00C0E0121210D0E02401F9D0E03400FAD052
:10134B00E0FBE50A0460DCD50AD980877BFF7A14C1
:10135B007965D202809C791080027908C206C20896
:10136B008008D2D5790A8004790AC2D5E50A0470BF
:10137B0002F50AE4FAFDFEFF1211CDFC7B082001F9
:10138B00131211CDFD7B1030000A1211CDFE12117C
:10139B00CDFF7B20EC3382D592D55013C3E43000C4
:1013AB00069FFFE49EFEE42001039DFDE49CFCE40C
:1013BB00CBF8C201EC700CCFCECDCCE824F8F87092
:1013CB00F38017C3EF33FFEE33FEED33FDEC33FC4D
:1013DB00EB33FB994002FB0FD8E9EB300105F8D05A
:1013EB00E0C448B201C0E00AEC4D4E4F78207B00C0
:1013FB0070C2EAB50A0040BCC0E012146BD0F0D04A
:10140B00E0200104C4C0E0C4B201C0F01211F9D055
:10141B00F0D5F0EB02124A12069012E75313615803
:10142B0012B84C12B44213654F136D44136D49122D
:10143B00CD4313735513574613574513574715137E
:10144B005012BC2D12C02E12E32B12C42312E1201A
:10145B0014FC2A127C48000012DB3F3F3F00790A44
:10146B00A2D5200314300509B910020404B90801F0
:10147B0004A2D52006025001042002689202B5098D
:10148B00005034C0E07F203003197F30A202720677
:10149B007205500F1214C2C202C206C205C2087FE7
:1014AB0030800F300503E9C0E0121210300503D075
:1014BB00E0F9D0E0B509CC3005177F30B9100C122C
:1014CB0012107F583004077F788003B9080312127B
:1014DB00103002057F2D0212107F202008F87F2B81
:1014EB002006F322920280CF286E756C6C2900D2F5
:1014FB00011211CD3001F8C201780930D50108F67F
:10150B0002127C2D504349581211CD2403B405000F
:10151B004001E490150E93121201743A121201D28B
:10152B0003750904021361900512EFF09004841205
:10153B00063712011CFF900512E0FEEE6F600302EE
:10154B0017559004841206377582027583001201B9
:10155B0035FFEF120690157410158E2016513016AC
:10156B007B401735500000174743BA805391FB530C
:10157B0092FBB29212255343BA805391FB5392FBC9
:10158B00B29222900484120637758205758300127D
:10159B000135FFEFC39403400302175590048412E7
:1015AB000637758206758300120135FF7E00EF7FCB
:1015BB0000FE9004841206377582077583001201B2
:1015CB0035FD7C00EE4CFEEF4DFF90048412063788
:1015DB00758205758300120135FDED25E025E024AC
:1015EB0008F582E43402F583EEF0A3EFF0900223CA
:1015FB001205439004841206377582057583001219
:10160B000135FDED25E025E0240AF582E43402F5F1
:10161B0083EEF0A3EFF043BA805391FB5392FBB2EE
:10162B009212291843BA805391FB5392FBB2921238
:10163B0027F97B017A027976900453743AF07F0094
:10164B007E00122E672290023EE0FEA3E0FF900286
:10165B0040EEF0A3EFF043BA805391FB5392FBB2F1
:10166B0092122A2543BA805391FB5392FBB29222DA
:10167B0090031FE4F090031FE0FFEFC394034003BC
:10168B000217557F0012203B7BFF7A2F794C90037A
:10169B001FE0FF7E009002ABEEF0A3EFF090031F74
:1016AB00E0FFEF25E025E02408F582E43402F58322
:1016BB00E0FEA3E0FF9002ADEEF0A3EFF090031F6E
:1016CB00E0FFEF25E025E02408F582E43402F58302
:1016DB00E0FEA3E0FF9002AFEEF0A3EFF090031F4C
:1016EB00E0FFEF25E025E0240AF582E43402F583E0
:1016FB00E0FEA3E0FF9002B1EEF0A3EFF090031F2A
:10170B00E0FFEF25E025E0240AF582E43402F583BF
:10171B00E0FEA3E0FF9002B3EEF0A3EFF01212385D
:10172B0090031FE004F0021680227F0012203B7B07
:10173B00FF7A2F79671212381222F0227F001220C3
:10174B003B7BFF7A2F796E1212382290036BEFF0EE
:10175B0090036C12065790036BE0FF12203B900333
:10176B006BE0FF121E2E90036BE0FFEF75F019A4D8
:10177B002424F582E43401F583E0FEA3E0FF7C0032
:10178B007D031201DB90036FE0FCA3E0FDD3ED9F23
:10179B00EC9E402F90036BE0FFEF75F019A424240F
:1017AB00F582E43401F583E0FEA3E0FF7C007D03CA
:1017BB001201DBEF24FFFFEE34FFFE90036FEEF020
:1017CB00A3EFF0900371E4F0A3E4F090036FE0FE5D
:1017DB00A3E0FF900371E0FCA3E0FDC3ED9FEC9E43
:1017EB0040030218F8900371E0FEA3E0FF7C007D3C
:1017FB00031201C9900373EEF0A3EFF090036C1288
:10180B000637900371E0FEA3E0FF8F828E831201F7
:10181B0035FFEFC4540FFFEF25E02412F582E434BB
:10182B0037F583E493FF90036BE0FEEE75F019A49C
:10183B002421F582E43401F583120637900373E01B
:10184B00FCA3E0FD8D828C83EF1201A7900373E460
:10185B0075F00112026690036C120637900371E06B
:10186B00FEA3E0FF8F828E83120135FFEF540FFF33
:10187B00EF25E02412F582E43437F583E493FF90EF
:10188B00036BE0FEEE75F019A42421F582E434011C
:10189B00F583120637900373E0FCA3E0FD8D828C79
:1018AB0083EF1201A7900373E475F00112026690A7
:1018BB00036BE0FFEF75F019A42421F582E43401EA
:1018CB00F583120637900373E0FEA3E0FF8F828E41
:1018DB008374201201A7900373E475F00112026662
:1018EB00900371E475F0011202660217D690036B38
:1018FB00E0FFEF75F019A42421F582E43401F583A0
:10190B00120637900373E0FEA3E0FF8F828E837481
:10191B00201201A7900373E475F001120266900385
:10192B006BE0FFEF75F019A42421F582E43401F587
:10193B0083120637900373E0FEA3E0FF8F828E8342
:10194B00E41201A790036BE0FF900373E0FCA3E0AC
:10195B00FDED24FFFDEC34FFFC12221E229005242A
:10196B00EFF0900524E0FFEF75F00EA42403F58251
:10197B00E43400F583E0FFEF6003021A4690052480
:10198B00E0FFEF75F00EA42403F582E43400F58339
:10199B007401F0900524E0FFEF75F00EA42404F51C
:1019AB0082E43400F583E4F0A3E4F0900524E0FF37
:1019BB00EF75F00EA42406F582E43400F583E4F011
:1019CB00900524E0FFEF75F00EA4240AF582E434B1
:1019DB0000F583E4F0900524E0FFEF75F00EA424EE
:1019EB0000F582E43400F583E0FF900524E0FEEE81
:1019FB0075F00EA4240BF582E43400F58312063740
:101A0B00900524E0FEEE75F00EA42404F582E43478
:101A1B0000F583E0FCA3E0FD8D828C83EF1201A720
:101A2B00900524E0FFEF75F00EA42404F582E43456
:101A3B0000F583E475F00112026622900524E0FFA5
:101A4B00EF75F00EA42400F582E43400F583E0FF7B
:101A5B00900524E0FEEE75F00EA4240BF582E43421
:101A6B0000F583120637900524E0FEEE75F00EA408
:101A7B002404F582E43400F583E0FCA3E0FD8D82C1
:101A8B008C83EF1201A7900524E0FFEF75F00EA4F5
:101A9B002404F582E43400F583E475F00112026648
:101AAB00900524E0FFEF75F00EA42404F582E434D6
:101ABB0000F583E0FEA3E0FF900524E0FEEE75F059
:101ACB000EA4240AF582E43400F583EFF09005248C
:101ADB00E0FFEF75F00EA42408F582E43400F583E3
:101AEB00E0FEA3E0FF900524E0FDED75F00EA424CD
:101AFB0004F582E43400F583E0FCA3E0FDC3ED9F25
:101B0B00EC9E4059900524E0FFEF75F00EA42406DF
:101B1B00F582E43400F5837402F0900524E0FFEFC6
:101B2B0075F00EA42407F582E43400F5837401F0FC
:101B3B00900524E0FFEF75F00EA42403F582E43446
:101B4B0000F583E4F0900524E0FFEF75F00EA4247C
:101B5B0004F582E43400F583E4F0A3E4F022900270
:101B6B009EE0FEA3E0FFE4FCFD90022312055FD391
:101B7B0012047E4003021C2A90029AE0FEA3E0FFAF
:101B8B00E4FCFD90022312055FD312047E501190EA
:101B9B00029AE0FEA3E0FFE4FCFD9002231205E0B5
:101BAB0090029AE0FEA3E0FFAB07AA06E4F9F890D7
:101BBB00022312054312032F9002331205E0900209
:101BCB009AE0FEA3E0FF90029EE0FCA3E0FDC3EDD4
:101BDB009FFFEC9EFEE4FCFD9002371205E09002A5
:101BEB003312055F900298E0FEA3E0FF90029CE0A9
:101BFB00FCA3E0FDC3ED9FFFEC9EFEE4FCFD120396
:101C0B003D9002331205E0900233120543900237E8
:101C1B0012055F1203C89002331205E0021CC0903C
:101C2B00029EE0FEA3E0FFAB07AA06E4F9F89002E0
:101C3B002312054312032F9002331205E090029EEC
:101C4B00E0FEA3E0FF9002A2E0FCA3E0FDC3ED9F4A
:101C5B00FFEC9EFEE4FCFD9002371205E090023390
:101C6B0012055F90029CE0FEA3E0FF9002A0E0FC57
:101C7B00A3E0FDC3ED9FFFEC9EFEE4FCFD12033DD4
:101C8B009002331205E09002331205439002371293
:101C9B00055F1203C89002331205E0900233120560
:101CAB005F90029CE0FEA3E0FFE4FCFD1203229098
:101CBB0002331205E090023312054390023EEEF020
:101CCB00A3EFF0229003E8EFF09003E91206579090
:101CDB0003E8E0FF12203B9003E8E0FF7D011231A7
:101CEB00629003E8E0FFEF75F019A42420F582E47D
:101CFB003401F5837401F09003E8E0FFEF75F01900
:101D0B00A4241CF582E43401F5831205EC000000D9
:101D1B00009003E8E0FFEF75F019A42417F582E4B7
:101D2B003401F583E4F0A37401F09003E8E0FFEFD6
:101D3B0075F019A42424F582E43401F583E0FEA3A5
:101D4B00E0FF9003ECE0FCA3E0FDD3ED9FEC9E40A5
:101D5B00289003E8E0FFEF75F019A42424F582E442
:101D6B003401F583E0FEA3E0FFEF24FFFFEE34FF29
:101D7B00FE9003ECEEF0A3EFF09003ECE0FEA3E09B
:101D8B00FF9003E8E0FDED75F019A42419F582E44A
:101D9B003401F583EEF0A3EFF09003EEE4F0A3E44F
:101DAB00F09003ECE0FEA3E0FF9003EEE0FCA3E079
:101DBB00FDC3ED9FEC9E50489003E912063790034C
:101DCB00EEE0FEA3E0FF8F828E83120135FF9003BE
:101DDB00E8E0FEEE75F019A42421F582E43401F558
:101DEB00831206379003EEE0FCA3E0FD8D828C831B
:101DFB00EF1201A79003EEE475F00112026680A1C9
:101E0B009003E8E0FFEF75F019A42421F582E43488
:101E1B0001F58312063712011CFD9003E8E0FF1257
:101E2B00331422900519EFF0900519E0FFEF75F0D0
:101E3B0019A42419F582E43401F583E4F0A3E4F04A
:101E4B00900519E0FFEF75F019A42417F582E4341F
:101E5B0001F583E4F0A3E4F0900519E0FFEF75F0D2
:101E6B0019A42420F582E43401F5837401F0900564
:101E7B0019E0FFEF25E02431F582E43437F583E4F4
:101E8B0093FE740193FF900519E0FDED75F019A415
:101E9B002424F582E43401F583EEF0A3EFF09005F2
:101EAB0019E0FFEF1206901EC2001EDF011EFC029E
:101EBB001F190300001F357B017A007992900519D9
:101ECB00E0FFEF75F019A42421F582E43401F583CA
:101EDB00120657227B017A017912900519E0FFEF68
:101EEB0075F019A42421F582E43401F58312065709
:101EFB00227B017A017913900519E0FFEF75F01938
:101F0B00A42421F582E43401F583120657227B01C8
:101F1B007A017914900519E0FFEF75F019A42421CB
:101F2B00F582E43401F5831206572290048CEFF00E
:101F3B0090048DECF0A3EDF090048CE0FF12203BAD
:101F4B0090048DE0FEA3E0FF90048FEEF0A3EFF082
:101F5B0090048FE0FFEFC4540FFFEF25E02412F540
:101F6B0082E43437F583E493FF90048CE0FEEE7546
:101F7B00F019A42426F582E43401F583EFF09004E4
:101F8B008FE0FFEF540FFFEF25E02412F582E434CE
:101F9B0037F583E493FF90048CE0FEEE75F019A403
:101FAB002427F582E43401F583EFF0900490E0FFF1
:101FBB00EFC4540FFFEF25E02412F582E43437F51C
:101FCB0083E493FF90048CE0FEEE75F019A42428B3
:101FDB00F582E43401F583EFF0900490E0FFEF54C9
:101FEB000FFFEF25E02412F582E43437F583E493F9
:101FFB00FF90048CE0FEEE75F019A42429F582E421
:10200B003401F583EFF090048CE0FF7E19EF8EF036
:10201B00A4FFAEF074262FF974013EFA7B019004F5
:10202B008CE0FF9003ECE4F0A37404F0121CCF22BD
:10203B00900517EFF0900517E0FFEF75F019A4244A
:10204B001CF582E43401F5831205EC0000000090CE
:10205B000517E0FFEF75F019A42417F582E434019E
:10206B00F583E0FEA3E0FFEF4E70030221369005EF
:10207B0017E0FFEF75F019A4241CF582E43401F589
:10208B00831205437B017A007900780012032290BA
:10209B000517E0FBEB75F019A4241CF582E4340161
:1020AB00F5831205E0900517E0FFEF75F019A424F6
:1020BB001CF582E43401F5831205437B207A4E79BB
:1020CB00007800C312047E5086900517E0FFEF7571
:1020DB00F019A42417F582E43401F583E0FEA3E0A4
:1020EB00FF900517E0FDED75F019A42419F582E4B6
:1020FB003401F583EEF0A3EFF0900517E0FFEF75D9
:10210B00F019A42420F582E43401F5837401F090D6
:10211B000517E0FFEF75F019A42417F582E43401DD
:10212B00F583E4F0A3E4F02202205A229004DE129D
:10213B0006579004DE120637758202758300120271
:10214B00BDFFAEF09004DE120637120292FDACF02A
:10215B00C3EF9DEE9C404D9004DE12063775820452
:10216B007583001202BDFFAEF09004DE12063775C8
:10217B0082027583001202BDFDACF0D3ED9FEC9E85
:10218B00500302221D9004DE120637120292FFAE9C
:10219B00F09004DE120637758202758300EE8FF025
:1021AB001202F5229004DE12063775820275830047
:1021BB001202BDFFAEF09004DE120637120292FD42
:1021CB00ACF0C3EF9DEE9C50499004DE12063775C0
:1021DB0082047583001202BDFFAEF09004DE12067E
:1021EB00377582027583001202BDFDACF0C3ED9F03
:1021FB00EC9E501E9004DE120637120292FFAEF0D8
:10220B009004DE120637758202758300EE8FF01292
:10221B0002F5229004C9EFF09004CAECF0A3EDF0A4
:10222B009004C9E0FF12203B9004C9E0FF7D01122E
:10223B0031629004C9E0FF121E2E9004C9E0FFEF3B
:10224B0075F019A42424F582E43401F583E0FEA390
:10225B00E0FF9004CAE0FCA3E0FDD3ED9FEC9E40B1
:10226B00289004C9E0FFEF75F019A42424F582E44B
:10227B003401F583E0FEA3E0FFEF24FFFFEE34FF14
:10228B00FE9004CAEEF0A3EFF09004CAE0FEA3E0C8
:10229B00FF9004C9E0FDED75F019A42419F582E453
:1022AB003401F583EEF0A3EFF09004C9E0FFEF7576
:1022BB00F019A42417F582E43401F583E4F0A37438
:1022CB0001F09004C9E0FFEF75F019A42421F58209
:1022DB00E43401F58312063712011CFD9004C9E0AA
:1022EB00FF1233142290015EE0FCA3E0FD7F00128D
:1022FB001F367D097F0012365F90018CE0FCA3E056
:10230B00FD7F00121F367D097F0012365F9001BAE8
:10231B00E0FCA3E0FD7F00121F367D097F00123623
:10232B005F9001E8E0FCA3E0FD7F00121F367D0902
:10233B007F0012365F7D7C7F0012365F7D097F0048
:10234B0012365F900223120543AD07AC067F0012D5
:10235B001F367D097F0012365F7F0012203B7BFF0B
:10236B007A2F797B90023EE0FEA3E0FF9002ABEE6A
:10237B00F0A3EFF090023EE0FEA3E0FF9002ADEE83
:10238B00F0A3EFF01212387F0012203B7BFF7A2F65
:10239B007985900242E0FEA3E0FF9002ABEEF0A342
:1023AB00EFF0900242E0FEA3E0FF9002ADEEF0A34F
:1023BB00EFF01212382290031FE4F090031FE0FF9E
:1023CB00EFC39404400302245990031FE0FF7E08DF
:1023DB00EF8EF0A4FFAEF0742E2FF974013EFA7B52
:1023EB0001C003C002C00190031FE0FF7E08EF8E07
:1023FB00F0A4FFAEF074762FF974023EFA7B0190D5
:10240B00038C12065790038FE4F0A37408F0D001ED
:10241B00D002D003122FF390031FE0FF7E08EF8E44
:10242B00F0A4FFAEF0742E2FF974013EFA7B0190ED
:10243B00031FE0FFEF75F02EA42454F582E4340162
:10244B00F58312065790031FE004F00223C67B01AD
:10245B007A027906C003C002C0017B017A02799629
:10246B0090038C12065790038FE4F0A37410F0D0F6
:10247B0001D002D003122FF37B017A02790690026E
:10248B001C12065722900513E4F07B017A02797631
:10249B0090045A743AF07F007E001230AE7F001227
:1024AB00203B7BFF7A367917900513E0FF7E009077
:1024BB0002ABEEF0A3EFF01212387B017A027976C1
:1024CB0090036FE4F0A3743AF07F0012175690025A
:1024DB00A6E0FEA3E0FFEFB4551DEEB4AA1912233C
:1024EB00C17F0012203B7BFF7A3679251212389080
:1024FB000513E0FF22803E9002A674AAF0A3745548
:10250B00F07F0012203B7BFF7A3679319002A6E0F8
:10251B00FEA3E0FF9002ABEEF0A3EFF01212381225
:10252B0027F97B017A027976900453743AF07F0095
:10253B007E00122E67900513E0FF04F0EFC39402A8
:10254B0050030224957F64229004E7740CF09004EE
:10255B00E87412F090024474AAF09002457402F0F1
:10256B009002467410F09004E7E0FF7F00EF54FFF9
:10257B00FF900247EFF09004E7E0FFEF54FFFF906E
:10258B000248EFF090015EE0FEA3E0FF900249EEFF
:10259B00F0A3EFF090018CE0FEA3E0FF90024BEE76
:1025AB00F0A3EFF09001BAE0FEA3E0FF90024DEE36
:1025BB00F0A3EFF09001E8E0FEA3E0FF90024FEEF6
:1025CB00F0A3EFF0900242E0FEA3E0FF900251EE89
:1025DB00F0A3EFF0900223120543900253EEF0A309
:1025EB00EFF09002557433F07B017A02794490043A
:1025FB00E8E0FF7E009003ECEEF0A3EFF07F00121B
:10260B001CCF22C0E0C0F0C083C082C0D075D00008
:10261B00C000C001C002C003C004C005C006C00793
:10262B00309817C298900000E599F0900002E4F002
:10263B00900001E4F07F00121968309954C2999010
:10264B000117E0FEA3E0FF900119E0FCA3E0FDED14
:10265B006F7002EC6E602490012112063790011707
:10266B00E0FEA3E0FF8F828E83120135FF8F9990DE
:10267B000117E475F00112026680169001207401B7
:10268B00F0900119E4F0A3E4F0900117E4F0A3E457
:10269B00F0D007D006D005D004D003D002D001D0A3
:1026AB0000D0D0D082D083D0F0D0E0329003CDEFE9
:1026BB00F09003CE1206579003D1E4F09003D212A0
:1026CB0005EC000000009003D1E4F09003D1E0FF93
:1026DB00EFC3941850549003CDE0FF7D01122AA84C
:1026EB009003D212054378011204A29003D2120573
:1026FB00E09003CDE0FF7D00122AA89003CDE0FF10
:10270B0012310AEF601C9003D2120543EF2401FF34
:10271B00EE3400FEED3400FDEC3400FC9003D212DD
:10272B0005E09003D1E004F080A19003CDE0FF7DA4
:10273B0001122AA89003CDE0FF7D00122AA8900376
:10274B00D21205439003CE12063712050522787F6D
:10275B00E4F6D8FD9000007F207E04E4F0A3DFFCBC
:10276B00DEFA750D00750E007581210227B4022B60
:10277B002BE493A3F8E493A34003F68001F208DF64
:10278B00F48029E493A3F85407240CC8C333C4542E
:10279B000F4420C8834004F456800146F6DFE480E2
:1027AB000B0102040810204080902CA5E47E0193BD
:1027BB0060BCA3FF543F30E509541FFEE493A360B4
:1027CB00010ECF54C025E060A840B8E493A3FAE40F
:1027DB0093A3F8E493A3C8C582C8CAC583CAF0A360
:1027EB00C8C582C8CAC583CADFE9DEE780BE9003CD
:1027FB001FE4F090031FE0FFEFC3940450569003C7
:10280B001FE0FF7E08EF8EF0A4FFAEF074762FF979
:10281B0074023EFA7B01C003C002C00190031FE0AB
:10282B00FF7E08EF8EF0A4FFAEF0742E2FF974012B
:10283B003EFA7B0190038C12065790038FE4F0A3B2
:10284B007408F0D001D002D003122FF390031FE0D5
:10285B0004F0809F7B017A027996C003C002C0010D
:10286B007B017A02790690038C12065790038FE452
:10287B00F0A37410F0D001D002D003122FF3220D6D
:10288B000A4144435F53414D504C4520696E697476
:10289B0020636828256429202020000D0A20445F2E
:1028AB004144435F4A49545445525F7A65726F2DD8
:1028BB002D2D000D0A20636828256429206164638F
:1028CB003D253564092D3E6F66667365742025358D
:1028DB00642077616E746C696E6520253564200009
:1028EB000D0A20636828256429206164633D253522
:1028FB0058092D3E6F666673657420253558207711
:10290B00616E746C696E652025355820009004E962
:10291B00740CF09004EA7412F090025874AAF090C0
:10292B0002597402F090025A7420F09004E9E0FF0F
:10293B007F00EF54FFFF90025BEFF09004E9E0FFA4
:10294B00EF54FFFF90025CEFF07B017A02795DC0E0
:10295B0003C002C0017B017A02799890038C1206A6
:10296B005790038FE4F0A3740CF0D001D002D00386
:10297B00122FF39002697433F07B017A027958902D
:10298B0004EAE0FF7E009003ECEEF0A3EFF07F0093
:10299B00121CCF22900522EFF043BA8053C9DF53AC
:1029AB00CADF43BA8053917F53927FC2977F021243
:1029BB00363B43BA804391405392BF43BA8053B1E5
:1029CB00FB53B2FBC2B27F0212363B43BA8043B118
:1029DB000853B2F743BA8053B1EF53B2EFC2B47F8F
:1029EB000212363B43BA8043B12053B2DF43BA8065
:1029FB0053B1BF53B2BFC2B67F0212363B43BA804C
:102A0B0043B18053B27F43BA8053C9EF53CAEFD25D
:102A1B00CC900522E0FF122D8F229004EB7402F074
:102A2B009004EC7408F090026C74AAF090026D7430
:102A3B0002F090026E7430F09004EBE0FF7F00EF39
:102A4B0054FFFF90026FEFF09004EBE0FFEF54FFA9
:102A5B00FF900270EFF0900240E0FEA3E0FFEEFF6C
:102A6B007E00EF54FFFF900271EFF0900240E0FE0A
:102A7B00A3E0FFEF54FFFF900272EFF0900273742C
:102A8B0033F07B017A02796C9004ECE0FF7E0090CE
:102A9B0003ECEEF0A3EFF07F00121CCF2290050B9E
:102AAB00EFF090050CEDF090050BE0FFEF120690A8
:102ABB002ACB002AE3012AFB022B130300002B2A4B
:102ACB0090050CE0FFEF6008D2977F0112363B2296
:102ADB00C2977F0212363B2290050CE0FFEF600895
:102AEB00D2B27F0112363B22C2B27F0212363B2298
:102AFB0090050CE0FFEF6008D2B47F0112363B2249
:102B0B00C2B47F0212363B2290050CE0FFEF600847
:102B1B00D2B67F0112363B22C2B67F0212363B225F
:102B2B0090034BE4F0A3E4F07BFF7A3179EEC00322
:102B3B00C002C0017B017A03794DA801AC02AD0341
:102B4B00D001D002D0037E007F091200F6122DFEB9
:102B5B0012000E9002D0120543EF240AFFEE340050
:102B6B00FEED3400FDEC3400FC9002D81205E07F42
:102B7B000012203B7BFF7A3179DC1212389002DC99
:102B8B00E0FFEFB401059002DCE4F0123596EF6044
:102B9B00057FAA1215327B017A027916120E3D803F
:102BAB00DC22900469EEF0A3EFF090046BECF0A341
:102BBB00EDF090046BE0FEA3E0FFEE30E73A9004FB
:102BCB006BE0FEA3E0FFC374FF9FFF74FF9EFE90BC
:102BDB00046BEEF0A3EFF090046BE0FEA3E0FF902C
:102BEB000469E0FCA3E0FDC3ED9FFFEC9EFE9004A7
:102BFB006DEEF0A3EFF0801E900469E0FEA3E0FF02
:102C0B0090046BE0FCA3E0FDED2FFFEC3EFE900487
:102C1B006DEEF0A3EFF090046DE0FEA3E0FF2290C9
:102C2B000514EFF0900514E0FF7E2EEF8EF0A4FF5D
:102C3B00AEF0744E2FF974013EFA7B0112352E90D3
:102C4B000514E0FFEF75F02EA42452F582E4340155
:102C5B00F58374E0F0900514E0FF7E08EF8EF0A48E
:102C6B00FFAEF0742E2FF974013EFA7B0190051420
:102C7B00E0FFEF75F02EA42454F582E43401F583C4
:102C8B00120657900514E0FFEF75F02EA42457F5AC
:102C9B0082E43401F5837401F0225002065745009B
:102CAB000018D900C81C2C035226F94109602001D9
:102CBB002E410018DA19630205410118DA192702AF
:102CCB0005410218DA18360205410318DA18F0022A
:102CDB000559011500000000000000000000000075
:102CEB00000000000000000000000000004E00008B
:102CFB000000000000000000000000000000460380
:102D0B002000000000000043048100000043048405
:102D1B000000000090046FEEF0A3EFF0900471EC54
:102D2B00F0A3EDF0900471E0FEA3E0FFEE30E72C92
:102D3B00900471E0FEA3E0FFC374FF9FFF74FF9E3E
:102D4B00FE900473EEF0A3EFF090046FE0FEA3E0AF
:102D5B00FF900473EE8FF0120266801F900471E0F7
:102D6B00FEA3E0FF90046FE0FCA3E0FDC3ED9FFF2B
:102D7B00EC9EFE900473EEF0A3EFF0900473E0FE74
:102D8B00A3E0FF22900521EFF0900521E0FFEF1269
:102D9B0006902DAA002DF5012DF84000002DFB43C8
:102DAB00BA8043918053927F43BA804391405392B0
:102DBB00BF43BA8043B10453B2FB43BA8043B1085B
:102DCB0053B2F743BA8043B11053B2EF43BA8043C7
:102DDB00B12053B2DF43BA8043B14053B2BF43BAC1
:102DEB008043B18053B27FC2CC22D2CD22C2CD223E
:102DFB00C2CD229004EDE4F0A3E4F07FC87E001274
:102E0B00345612349090FE01E4F01236AD120003EA
:102E1B001231F71236BED2A97F0012203B7BFF7A0C
:102E2B003179B99002AB1205EC01518000121238C6
:102E3B001224907E009004EDEEF0A3EFF07F0012D1
:102E4B00203B7BFF7A3179CD9004EDE0FEA3E0FFD0
:102E5B009002ABEEF0A3EFF01212382290044EEE7C
:102E6B00F0A3EFF0900450120657900454E4F09046
:102E7B00044EE0FEA3E0FF1234FA900454E4F09009
:102E8B000453E0FF900454E0FEEEC39F50349004D3
:102E9B0054E0FF7E0090044EE0FCA3E0FDEF2DFF1D
:102EAB00EE3CFE900450120637900454E0FD8D82E8
:102EBB00758300120135FD12339A900454E004F02F
:102ECB0080BD229002D01205437B017A00790078F5
:102EDB00001203229002D01205E07B507A00790099
:102EEB0078009002D01205431203C8AC00AD01AEBE
:102EFB0002AF037B007A0079007800C312047E7066
:102F0B001D9002D41205437B017A007900780012E0
:102F1B0003229002D41205E09002DC7401F09002BF
:102F2B00DE1206371206B622204C335F7461736BC8
:102F3B005F7765696768745F68616E646C65722042
:102F4B00000D0A25643A202534782825346420297D
:102F5B002025347828253664290D0A000D0A20090E
:102F6B00090900207070206572726F720D0A2000C3
:102F7B00202825642925347820006F757420282596
:102F8B0064292534780D0A009004E4E4F09004E5FC
:102F9B00E4F09004E6E4F090000B12063712011CEB
:102FAB00FF9004E4EFF090000B1206377582017569
:102FBB008300120135FF9004E5EFF090000B120631
:102FCB0037758202758300120135FF9004E6EFF02E
:102FDB009004E4E0FFEFB4AA0C9004E5E0FFEFB43B
:102FEB0002037F01227F0022900389120657900370
:102FFB0091E4F0A3E4F090038FE0FEA3E0FF9003D5
:10300B0091E0FCA3E0FDC3ED9FEC9E503890038C48
:10301B00120637900391E0FEA3E0FF8F828E83129E
:10302B000135FF900389120637900391E0FCA3E072
:10303B00FD8D828C83EF1201A7900391E475F00153
:10304B0012026680B122900523EFF0900523E0FF7A
:10305B00EF75F00EA42406F582E43400F583E4F05A
:10306B00900523E0FFEF75F00EA42407F582E434FE
:10307B0000F583E4F0900523E0FFEF75F00EA42438
:10308B0003F582E43400F583E4F0900523E0FFEFD1
:10309B0075F00EA42404F582E43400F583E4F0A368
:1030AB00E4F022900455EEF0A3EFF09004571206D3
:1030BB005790045BE4F090045BE4F090045AE0FF5B
:1030CB0090045BE0FEEEC39F503490045BE0FF7E08
:1030DB0000900455E0FCA3E0FDEF2DFFEE3CFE124B
:1030EB0033DA90045712063790045BE0FE8E82753C
:1030FB008300EF1201A790045BE004F080BD2290E7
:10310B00050DEFF090050E7409F090050DE0FFEF43
:10311B00120690312E00313A013146023152030032
:10312B0000315CA296E433FF90050EEFF08022A2F3
:10313B00B3E433FF90050EEFF08016A2B5E433FF36
:10314B0090050EEFF0800AA2B7E433FF90050EEF67
:10315B00F090050EE0FF229004FBEFF09004FCEDE5
:10316B00F09004FCE0FFEF701F9004FBE0FFEF1208
:10317B00069031AC0031AC0131AC0231AC03000034
:10318B0031AC2222222222229004FBE0FFEF120616
:10319B009031AC0031AC0131AC0231AC03000031E9
:1031AB00AC220D0A2025582025583A2558000D0A27
:1031BB00445F7379735F4D61696E46726509256C67
:1031CB0064000D0A4C335F535F696E6974092564A3
:1031DB00000D03206D61696E207768696C65313372
:1031EB000D0A00AB00000000000000007BFF7A32EC
:1031FB0079889002DE1206577BFF7A32798890022B
:10320B00E11206577BFF7A3279889002E11206575A
:10321B009002D41205EC000000009002D01205ECD5
:10322B00000000009002DCE4F07BFF7A327988909A
:10323B0002DE120657220D0A756172743120636C1F
:10324B006F7365000D0A7561727431206F70656E56
:10325B00000D0A7561727432206F70656E00323228
:10326B003A206D6F746F3D2825582900207070200F
:10327B006572726F720D0A200033333300900002B7
:10328B00E0FFEF703E900001E0FFEFC39402402D92
:10329B009000027401F0900003E4F090000AE0FF4C
:1032AB00EFD39400401790000AE4F09000067401ED
:1032BB00F07B017A00790E90000B120657900001FB
:1032CB00E004F0229004631205E0900463120543BE
:1032DB00780812048F9004631205E09004631205C2
:1032EB0043900467EEF0A3EFF0900467E0FEA3E0D9
:1032FB00FF7CFF7DFF1201C9900467EEF0A3EFF096
:10330B00900467E0FEA3E0FF229004F9EFF0900435
:10331B00FAEDF09004F9E0FFEF120690333700332B
:10332B003F01334702334F03000033569004FAE05A
:10333B00FF8F99229004FAE0FF8F9B229004FAE012
:10334B00FF8FAD229004FAE0FF8F8522C0E0C0F022
:10335B00C083C082C0D075D000C000C001C002C005
:10336B0003C004C005C006C007000000C28D122EAA
:10337B00CE000000D007D006D005D004D003D00279
:10338B00D001D000D0D0D082D083D0F0D0E032901A
:10339B0004D8EEF0A3EFF09004DAEDF075C780756A
:1033AB00F50C75C5029004D8E0FEA3E0FF8FC49026
:1033BB0004D8E0FEA3E0FFEEFF7E008FC39004DA9B
:1033CB00E0FF8FC275C65A75C6A5001236CF229084
:1033DB0004D5EEF0A3EFF075C78075F50C75C5013C
:1033EB009004D5E0FEA3E0FF8FC49004D5E0FEA3CC
:1033FB00E0FFEEFF7E008FC375C65A75C6A5009021
:10340B0004D7E5C2F01236CF9004D7E0FF227F003D
:10341B00121E2E7B017A00790E90000B120657902C
:10342B000008E4F0A37480F07F0012305143BA809F
:10343B0053B1FD53B2FD43BA8053B1FE53B2FE12EA
:10344B003681C298C299D29CD2AC229004BCEEF0C9
:10345B00A3EFF09004BCE0FEA3E0FF9004BEEEF0FF
:10346B00A3EFF09004BEE0FEA3E0FFD3EF9400EED9
:10347B00940040101235F09004BE74FF75F0FF12EB
:10348B00026680DF2243BA805391FB5392FBD292A8
:10349B0090031FE4F090031FE0FFEFC39406501A54
:1034AB0043BA805391FB5392FBB2927F2C7E011255
:1034BB00345690031FE004F080DB22900511EFF0EF
:1034CB00900511E0FFEF601A7F0112299F7F001218
:1034DB002C2A7F01122C2A7F02122C2A7F03122CFA
:1034EB002A227B017A02790690021C12065722903F
:1034FB000509EEF0A3EFF075C78075F50C75C503E4
:10350B00900509E0FEA3E0FF8FC4900509E0FEA340
:10351B00E0FFEEFF7E008FC375C65A75C6A500127D
:10352B0036CF229004DB1206579004DB1206377558
:10353B008204758300E41201A79004DB1206377531
:10354B008205758300E41201A79004DB1206371283
:10355B00061D000000002290049612065790049955
:10356B00E4F0A3E4F0900496E475F0011206401227
:10357B00011CFFEF600C900499E475F001120266D8
:10358B0080E3900499E0FEA3E0FF22900007E0FFA8
:10359B00EFB40105900007E4F0900006E0FFEFB4F4
:1035AB000115900006E4F07B017A00790E900484FB
:1035BB00120657122F93227F00229004A0EFF09057
:1035CB0004A11206579004A112063712356290031C
:1035DB00ECEEF0A3EFF09004A0E0FF9004A1120634
:1035EB0037121CCF229004F3741DF09004F3740A6D
:1035FB00F09004F47434F09004F4E014FFF0EF70E6
:10360B00F69004F3E014FFF0EF70EC220D0A7265F4
:10361B00616420533A20256409000D0A53706172CE
:10362B0061096F6B09000D0A50726F6720257800D6
:10363B009004F1EFF09004F1E0FF9004F2EFF090C2
:10364B0004F2E0FFEFD394004009009004F2E01481
:10365B00F080EC229004FDEFF09004FEEDF090046E
:10366B00FDE0FF7B017A0479FE9003ECE4F0A37498
:10367B0001F0121CCF22759850438E40538EFE538F
:10368B00890F758BC0758DFDC2ABD28E2290052B29
:10369B00EFF090052BE0FD7F0012365F90052BE0DD
:1036AB00FF22123419D2AF7BFF7A32794F7F00128F
:1036BB0035C522538E7F5389F0758A00758CA6C24F
:1036CB008DD28C2275C70075C50075C60075C38079
:1036DB0075C400220001000A006403E827100000F3
:1036EB0000010000000A00000064000003E8000075
:1036FB002710000186A0000F42400098968005F528
:10370B00E1003B9ACA00003001310232033304342A
:10371B00053506360737083809390A410B420C4381
:0E372B000D440E450F46008000010001000114
:00000001FF
